:100000000C94B2050C94CF050C94CF050C94142ECF
:100010000C94CF050C94CF050C94CF050C94CF0510
:100020000C94CF050C94CF050C9428160C94491A07
:100030000C941B260C94CF050C94CF050C94CF0583
:100040000C94CF050C94CF050C94CF050C94CF05E0
:100050000C94CF050C9401170C94CF050C94CF058C
:100060000C94CF050C94CF050C94CF050C94CF05C0
:100070000C94CF050C94CF050C94CF050C94CF05B0
:100080000C94CF050C94CF050C94CF050C94CF05A0
:100090000C94CF050C94CF050C94CF050C94CF0590
:1000A0000C94CF050C94CF050C94CF052020202074
:1000B0006162636465666768696A6B6C6D6E6F70B8
:1000C0007172737475767778797A31323334353664
:1000D00037383930524542545F2D3D5B5D5C233BE0
:1000E00027602C2E2F2020202B0014001A0008003F
:1000F00015001700E00004001600070009000A00C0
:10010000E1001D001B0006001900050000000000B2
:100110000000E300215228242900130012000C00E3
:1001200018001C00340033000F000E000D000B00FF
:10013000E500380037003600100011000000000014
:10014000000022522A002C2F01001E021F02200252
:100150002102220201001E001F00200021002200B7
:1001600001002300240025002600270000000000D5
:1001700000000100000001003100270226022502D4
:1001800024022302310230002F0035002E002D0002
:10019000010030022F0235022E022D020000000065
:1001A0000000010001000100007C3A003B003C001F
:1001B0003D003E000100AC00AB00AA00A900AE006B
:1001C0002078217823782578277829780000000086
:1001D0000000010000000100000027004200410073
:1001E00040003F00000000004F005200510050004E
:1001F00001000000000000000000000000000000FE
:10020000000000000100010000DA0281FFD9F1DBEB
:1002100020A4A62EAF00A0C0D30000A1C8D3000028
:10022000AED580A81F408D1420001E0F0500047F4E
:100230003F1F643214643214783C1E1E140A0555A4
:100240006E6465660041646A757374005261697317
:1002500065004C6F7765720044656661756C74006B
:100260004C617965723A20003A002C206B007800CE
:10027000808182838485868788898A8B8C8D8E8F06
:100280009091929394A0A1A2A3A4A5A6A7A8A9AA7D
:10029000ABACADAEAFB0B1B2B3B4C0C1C2C3C4C5F4
:1002A000C6C7C8C9CACBCCCDCECFD0D1D2D3D4004B
:1002B0000001010101010101010102020202020229
:1002C00002020203030303030303030404040404FC
:1002D00004040505050505060606060607070707C3
:1002E0000708080808090909090A0A0A0B0B0B0C78
:1002F0000C0C0D0D0D0E0E0E0F0F0F101011111115
:100300001212131314141515161617171818191995
:100310001A1A1B1B1C1D1D1E1E1F202021222223FA
:100320002424252626272829292A2B2C2D2D2E2F3B
:1003300030313232333435363738393A3B3C3D3E52
:100340003F404142434445464748494A4C4D4E4F41
:1003500050515354555658595A5B5D5E5F61626403
:10036000656668696B6C6D6F7072737577787A7B90
:100370007D7E8082838587888A8C8E8F91939596E7
:10038000989A9C9EA0A2A3A5A7A9ABADAFB1B3B507
:10039000B7BABCBEC0C2C4C6C9CBCDCFD1D4D6D8E3
:1003A000DBDDDFE2E4E7E9EBEEF0F3F5F8FAFDFF81
:1003B000FFAA7F55402223252628292A2C2D2F30BD
:1003C00032333536383A3B3D3E4042434547494A51
:1003D0004C4E5051535557595A5C5E606264666882
:1003E000696B6D6F71737577797B7D7F818385878D
:1003F000898A8C8E90929496989A9C9E9FA1A3A590
:10040000A7A8AAACAEAFB1B3B4B6B8B9BBBCBEBFB7
:10041000C1C2C3C5C6C7C9CACBCCCDCED0D1D2D23A
:10042000D3D4D5D6D7D7D8D9D9DADADBDBDBDCDC45
:10043000DCDCDCDDDDDDDDDCDCDCDCDCDBDBDBDAFD
:10044000DAD9D9D8D7D7D6D5D4D3D2D2D1D0CECD68
:10045000CCCBCAC9C7C6C5C3C2C1BFBEBCBBB9B875
:10046000B6B4B3B1AFAEACAAA8A7A5A3A19F9E9CFA
:100470009A98969492908E8C8A89878583817F7DC5
:100480007B79777573716F6D6B6968666462605EA6
:100490005C5A5957555351504E4C4A49474543426F
:1004A000403E3D3B3A3836353332302F2D2C2A2909
:1004B000282625232200AF00AE05010902A10185EF
:1004C000020901A100050919012908150025019556
:1004D00008750181020501093009311581257F95D3
:1004E000027508810609381581257F9501750881F7
:1004F00006050C0A38021581257F950175088106CD
:10050000C0C005010980A101850319012AB70015A2
:100510000126B700950175108100C0050C0901A1E5
:1005200001850419012AA002150126A00295017572
:10053000108100C005010906A1018506050719E023
:1005400029E71500250195087501810205071900A5
:1005500029EF1500250195F07501810205081901A3
:100560002905950575019102950175039101C00555
:10057000010906A101050719E029E71500250195E4
:100580000875018102950175088101050719002987
:10059000FF150026FF009506750881000508190162
:1005A0002905150025019505750191029501750331
:1005B0009101C009023B00020100A0FA09040000F9
:1005C0000103010100092111010001224400070576
:1005D0008103080001090401000103000000092152
:1005E0001101000122B6000705820320000112015B
:1005F0000002000000085346010001000102000152
:100600000C0343006F0072006E00650000001003D1
:1006100066006F006F007300740061006E000000E0
:10062000040309040000000000003E5B4F5B3E0035
:100630003E6B4F6B3E001C3E7C3E1C00183C7E3CDB
:1006400018001C577D571C001C5E7F5E1C000018A4
:100650003C180000FFE7C3E7FF0000182418000063
:10066000FFE7DBE7FF0030483A060E00262979292C
:100670002600407F05050700407F05253F005A3CC6
:10068000E73C5A007F3E1C1C0800081C1C3E7F00F3
:1006900014227F2214005F5F005F5F0006097F0164
:1006A0007F00006689956A0060606060600094A2C7
:1006B000FFA2940008047E04080010207E20100091
:1006C00008082A1C0800081C2A0808001E10101020
:1006D00010000C1E0C1E0C0030383E383000060E88
:1006E0003E0E060000000000000000005F00000059
:1006F000000700070000147F147F1400242A7F2ABB
:100700001200231308646200364956205000000886
:1007100007030000001C224100000041221C0000D1
:100720002A1C7F1C2A0008083E0808000080703040
:1007300000000808080808000000606000002010A1
:10074000080402003E5149453E0000427F4000003F
:100750007249494946002141494D33001814127F1E
:1007600010002745454539003C4A4949310041219F
:1007700011090700364949493600464949291E00F2
:1007800000001400000000403400000000081422A3
:100790004100141414141400004122140800020132
:1007A000590906003E415D594E007C1211127C0031
:1007B0007F49494936003E41414122007F41414144
:1007C0003E007F49494941007F09090901003E4136
:1007D000415173007F0808087F0000417F410000FD
:1007E0002040413F01007F08142241007F404040EB
:1007F00040007F021C027F007F0408107F003E4102
:1008000041413E007F09090906003E4151215E0039
:100810007F091929460026494949320003017F0111
:1008200003003F4040403F001F2040201F003F404A
:1008300038403F0063140814630003047804030085
:100840006159494D4300007F4141410002040810B5
:100850002000004141417F000402010204004040A9
:100860004040400000030708000020545478400036
:100870007F284444380038444444280038444428FD
:100880007F0038545454180000087E0902001824D0
:10089000241C78007F080404780000447D40000098
:1008A0002040403D00007F102844000000417F4070
:1008B00000007C04780478007C0804047800384444
:1008C000444438007C1824241800182424187C0080
:1008D0007C080404080048545454240004043F4491
:1008E00024003C4040207C001C2040201C003C4058
:1008F00030403C004428102844004C9090907C00EC
:100900004464544C44000008364100000000770065
:1009100000000041360800000201020402003C26EB
:1009200023263C0000000000000000000000000042
:1009300000000000C0E0F0F8F81800C0F0FCFEFF76
:10094000FFFFFFFFFFFF7E0000000000000000002F
:1009500080C0E0E0E0E0E0E0E0E0C0800000000017
:1009600080C0E0E0E0E0E0E0E0E0C080000000E027
:10097000E0C0C0E0E0E0E00000E0E0C0C0E0E0E0B7
:10098000E0E0C0800000000080C0E0E0E0E0E0E0E7
:10099000E0E0C08000000000000000000000000057
:1009A0000000E0F0F0F0E0ECEEF7F37020007C7C6B
:1009B0007C7E007E7E7E7F7F7F000080C0E07E5B4D
:1009C0004F5BFEC00000C000DCD7DEDEDED7DC00FF
:1009D000C000000000000000000000000000000057
:1009E00000000000000000000000000000F8FCFE15
:1009F000FFE000FFFFFFFFFFFF80FFFFFFFFFFFFA4
:100A0000FFFFFF1F0701000000000000000000FFC3
:100A1000FFFF8100000000000081C3C3C30000FF8E
:100A2000FFFF8100000000000081FFFFFF0000FFCA
:100A3000FFFF01000000000000FFFFFF01000000B9
:100A40000001FFFFFF0000FFFFFF9D1C1C1C1C1C82
:100A50001C9DDFDFDF000000000000000000000040
:100A600000000F1F3F7F7F7F7F7F3F1E0C001F1FF7
:100A70001F3F003F3F3F7F7F7F00307B7F783020EC
:100A80002030787F3B0003000F7F0F0F0F7F0F0098
:100A90000300000000000000000000000000000053
:100AA00000000000000000000000000000030F1F15
:100AB0003F3F3F3F1F1F3F3F7F7F7F3F3F1F3F7FA6
:100AC0007F7F7F7C7878381C0F00000000000000DA
:100AD00001030707070707070707030100000000D6
:100AE00001030707070707070707030100000007BF
:100AF00007070000000000000007070700000000D3
:100B000000000707070000000103070707070707A2
:100B100007070301000000000000000000000000C3
:100B200000000000000000000000000000000000C5
:100B300000000000000000000000000000000000B5
:100B400000000000000000000000000000000000A5
:100B50000000000000000000000000000000000095
:100B60000000000011241FBECFEFDAE0DEBFCDBFD2
:100B700027E0A6ECB1E001C01D92AA30B207E1F770
:100B800011E0A0E0B1E0EAE1F3E602C005900D92C9
:100B9000A63CB107D9F70E9442260C9437310C9439
:100BA0000000482F2091FB049091C20457E02913C4
:100BB00002C080E0089530E0529FF001539FF00D95
:100BC0001124ED53FB4F8181681306C080814813C7
:100BD00003C085818111EECF2F5F3F4F2770E7CF94
:100BE000FC01AC014C5F5F4F8FEF91E321918227B5
:100BF00028E030E087FF09C0880F8927215031099C
:100C0000C9F7E417F50791F70895880FF7CFE8EDD6
:100C1000F0E080818E7F80831092E2001092DA00F3
:100C20001092E100A0EEB0E08C9181608C93808105
:100C30008F77808319BCA7EDB0E08C918E7F8C9369
:100C400080818F7E80831092AB0408952091E40010
:100C50003091E50095E6A9012091EC00822F81708A
:100C600020FF06C08091E80080FF06C080E0089564
:100C70002091E80022FD1AC08091B804882389F0F1
:100C8000853089F08091EB0085FD0FC02091E40054
:100C90003091E50042175307F9F29150E1F684E0F4
:100CA000089582E0089583E0089581E00895809199
:100CB000BA0487FF13C08091E80082FF06C08091CC
:100CC000E8008B778093E80004C08091B80481111C
:100CD000F2CF08958091B8048823D9F38091E80079
:100CE00080FFF8CF8091E8008E77ECCF982F90931B
:100CF000E900242F762F50E0891731F07091EC0035
:100D00002091ED005091F00021FD07C09F5F9730CA
:100D100071F78093E90081E008953091EB003E7F08
:100D20003093EB003091ED003D7F3093ED0030913A
:100D3000EB0031603093EB007093EC002093ED00FA
:100D40005093F0002091EE0027FDE0CF80E0089561
:100D5000B0E0A0E0EEEAF6E00C944E2FC8EDD0E053
:100D600088818F7E8883E7EDF0E0808181608083D9
:100D700084E082BF81E08093AB0488818E7F88838A
:100D800002EE10E0F80110821092DA0081EEC82E17
:100D9000D12CF601108288818F77888388818068C2
:100DA000888388818F7D888319BC1092B804109243
:100DB000B9041092B7041092B60490EEE92EF12C0B
:100DC000F70180818B7F808388818160888342E006
:100DD00060E080E00E947606F60180818E7F80834D
:100DE000F801808181608083808188608083F70141
:100DF00080818E7F8083888180618883CDB7DEB7D4
:100E0000E8E00C946A2FFC018091C0049091C10429
:100E100086179707A0F06115710529F49091E800F5
:100E20009E779093E80090E06115710551F491115F
:100E300008C08091E80082FF34C080E00895BC01C2
:100E4000F2CF8091B8048823C1F18530C1F180913F
:100E5000E80083FD30C08091E80082FDEACF8091F8
:100E6000E80080FFE1CF8091F3002091F200382F5D
:100E70006115710519F02830310558F091E02830DE
:100E8000310509F090E02091E8002E772093E800EA
:100E9000CBCF81918093F100615071092F5F3F4F5B
:100EA000E7CF8091B804882341F0853041F08091EC
:100EB000E80083FFBECF81E0089582E0089583E0DB
:100EC00008958091AD04089587E797E7909301080E
:100ED0008093000888E19AE00FB6F894A895809373
:100EE00060000FBE90936000FFCF2FB7F894609121
:100EF000A7047091A8048091A9049091AA042FBF1F
:100F0000089590914C019923D1F09091A40497FFFA
:100F100016C0E82FE695E695E695EE31E0F4F0E0B0
:100F2000E053FE4F282F277081E090E001C0880F2A
:100F30002A95EAF780959281892382830895EAECC5
:100F4000F1E09191891303C0DF0111971C9291E0A8
:100F5000E03DF907B1F7089590914C019923C1F054
:100F60009091A40497FF14C0E82FE695E695E695C6
:100F7000EE31F8F4F0E0E053FE4F877021E030E00E
:100F800001C0220F8A95EAF78281822B828308951D
:100F9000AAECB1E0EFEF90E02D91821751F0EF3F16
:100FA00019F4211101C0E92F9F5F9630A9F7EF3F97
:100FB00009F408950E2E000CFF0BE853FE4FE6CF08
:100FC000A3E0B0E0E6EEF7E00C94542F2091A204E9
:100FD0003091A30428173907A1F09093A3048093BC
:100FE000A204E091A004F091A104309751F024E014
:100FF00029839B838A830084F185E02DCE010196AD
:1010000009952396E2E00C94702FA3E0B0E0EBE0AA
:10101000F8E00C94542F20919E0430919F042817DF
:101020003907A1F090939F0480939E04E091A0045F
:10103000F091A104309751F023E029839B838A83A8
:101040000084F185E02DCE01019609952396E2E01A
:101050000C94702F80919C04882359F0E091A00497
:10106000F091A104309729F00190F081E02D0995CD
:10107000089580E008958091910480FD16C081FD5F
:1010800016C082FD16C0809190048823A1F088329A
:1010900080F428E0829FC001112468E270E00E9481
:1010A000952F862F672B39F0089582E0089584E00C
:1010B000089588E0089581E008958091910480FD6D
:1010C00014C081FD14C082FD16C080918F04882356
:1010D00081F08E3180F420E5829FC00111246EE101
:1010E00070E00E94952F862F089584E1089588E28C
:1010F000089588E0089580E50895282F35EB2303AF
:10110000C001112497FF04C080589109892F0895C8
:1011100080589F4FFBCFFA01811101C0FB01099557
:1011200008950895EBECF2E011828281846082835D
:10113000089580918104982F9C7F61F4837084606E
:101140008093810480918404893718F088E7809324
:10115000840408958C3AB0F38370886AF1CFAF921B
:10116000BF92DF92EF92FF920F931F93CF93DF9383
:10117000182F062FE901493708F048E7E42FF0E07F
:10118000E055FD4F011110C0E4915E2F4E2F4983B1
:10119000E8835A83DF91CF911F910F91FF90EF90D9
:1011A000DF90BF90AF900895202F30E04491D42E6F
:1011B000E42EF12C56E0159FC0011124EFEFF0E072
:1011C000BF010E94302F812F90E0880F991F55E5B5
:1011D000569FD001579FB00D11248A1B9B0B982F4F
:1011E000990F890F5F01A21AB30AAE9CD001AF9C80
:1011F000B00DBE9CB00D11245B2F089F80011124FF
:10120000012F11275F01A01AB10AAE9C8001AF9C8B
:10121000100DBE9C100D11245F01A81AB108A29EEA
:10122000C001A39E900DB29E900D1124892F992785
:10123000E81BF90BEE9DC001EF9D900DFE9D900DFA
:101240001124E92F62307105A1F050F46115710588
:1012500009F49DCF6130710581F0EB2F512F97CFAD
:101260006430710569F080F06630710509F48FCF44
:10127000F4CFE42F4B2F592F8ACFE42F412F87CF64
:10128000EB2F542F492F83CF4B2F5D2DE12F7FCF95
:1012900080E00895F894E82FE295EF70F0E031A136
:1012A000282F2F7081E090E001C0880F2A95EAF77F
:1012B000982F9095932391A392A1892B82A3789440
:1012C00008950F931F9380919C04882329F00E9416
:1012D00075071F910F9108950E9475070091700284
:1012E000109171022091720230917302600F711F90
:1012F000821F931FEECF9091A40492FF10C041E093
:10130000282F2471243009F040E031E0282F287183
:10131000283009F030E0431711F02CE0822793FFCA
:1013200010C041E0282F2471243109F040E031E061
:10133000282F2871283109F030E0431711F02CE0F4
:1013400082273091A50430FF10C051E0282F217171
:10135000213009F050E041E0282F2871283009F0B1
:1013600040E0541711F029E0822731FF10C041E01E
:10137000282F2171213109F040E031E0282F287118
:10138000283109F030E0431711F029E0822794FD5D
:10139000877E089582389105B9F1B0F481339105C3
:1013A00009F47DC048F48932910509F46DC08A3290
:1013B000910509F47BC008958533910509F45FC058
:1013C0008933910509F10895833E9105D9F138F4E7
:1013D000803E910529F1823E910579F10895863E7E
:1013E0009105D9F1873E910509F43EC0843E9105EF
:1013F00041F52091A50421FF24C08091A40484FD1F
:1014000019C087EE90E008952091A404237009F09C
:101410005AC02091A50423FF14C089E290E00895EA
:101420002091A40420FD38C03091A50430FF09C0EC
:1014300024FF43C090E080E008952091A40422FDA1
:10144000F7CF08952091A40422FD3AC03091A5045D
:1014500030FD39C024FFF5CFEDCF2091A40423FF48
:10146000F0CF24FDE7CFCDCF2091A40423FD2EC0E3
:101470003091A50431FFEECF84EE90E008952091E5
:10148000A40425FFDECFC9CF2091A40425FD21C0EF
:101490002091A50423FFD5CF89E390E0D2CF2091FE
:1014A000A40426FFCECF8AE290E008952091A40400
:1014B00026FFC7CF81E390E0089583EE90E0089582
:1014C00082EE90E0089580EE90E0089586EE90E040
:1014D000089585E390E00895972F7830B8F466304A
:1014E000A8F48330B0F470E026E0929F600D711D87
:1014F0001124FB0190E3899FE00DF11D1124EE0FF3
:10150000FF1FE851FF4F85919491089580E090E08E
:10151000089581E0FCCF1F93CF93DF930E94CA0907
:10152000EC01C11580E5D807F0F5C11580E4D807B6
:1015300008F09CC0C03ED10520F5CD3CD10508F097
:1015400082C0C83AD10578F4C53AD10508F073C015
:10155000C130D10519F1209709F1C430D105F0F45B
:10156000D0E0C0E01BC0C33CD105D0F7C85AD0E0E2
:10157000CC0FDD1FC05BDE4F0990D881C02DD46435
:101580000DC0C11580E2D80708F0D1C0C11581E0B7
:10159000D80708F05AC0C83ED10510F7CE01DF9138
:1015A000CF911F910895C03682E5D80718F5C03451
:1015B00082E5D80708F06BC0C03282E5D80708F092
:1015C0005FC0C11582E5D80708F497C02C2F269577
:1015D000269580E2289F900111248C2F8370C1E012
:1015E000D0E002C0CC0FDD1F8A95E2F7C22BD32BCF
:1015F000DD68D4CFC03A82E5D80760F4C03882E510
:10160000D80708F459C0CF71D0E0DC2FCC27C46FC5
:10161000D06AC4CFC03C82E5D80708F462C0C03E9F
:1016200082E5D80708F09CCFDC2FCC27CC27DF71D0
:10163000C06FD06AB3CFC55AD0E0C35BDE4FC8815C
:10164000D0E0D064ABCFD065A9CF8D2F0E947B09AD
:10165000182FCE0199270E94CA09C12FD0E0DC2F94
:10166000CC27CC27DF71C82BD92B98CFCE01992757
:101670000E94CA09CC27DF70C82BD92BD06A8ECF25
:10168000CF71D0E0DC2FCC27C16FD06A87CF2C2F51
:1016900026952695277080E2289F900111248C2F93
:1016A0008370C1E0D0E002C0CC0FDD1F8A95E2F765
:1016B000C22BD32BDC6872CF2C2F26952695277052
:1016C00080E2289F900111248C2F8370C1E0D0E02C
:1016D00002C0CC0FDD1F8A95E2F7C22BD32BDA684C
:1016E0005DCF8C2F8F710E947B09C82FD0E0DC2F3B
:1016F000CC27CC27DF71D06251CF8C2F8F710E9405
:101700007B0955E0D695C7955A95E1F7CF70D0E0A3
:10171000DC2FCC27282F30E084FF05C044E0220FC7
:10172000331F4A95E1F7C22BD32BD06937CF8D2FCA
:101730008F710E947B09182FCE0199270E94CA0938
:10174000C12FD0E0DC2FCC27CC27DF71C82BD92BC1
:10175000D2CF809590913C02982390933C020895BB
:1017600080913C0290911302892B9091120299234F
:1017700091F0892B90914C01992371F09091A404E0
:1017800097FF0AC09EE122ED31E040E0915040F425
:10179000411110921202089596E02AEC31E0F5CF43
:1017A000F90151919F01552389F34F5FEFCF80914C
:1017B000FB049091C204981301C008958F5F877055
:1017C000FACFB0E0A0E0E7EEFBE00C944D2F7C01F7
:1017D000009193021091940280913D0290913E02FB
:1017E000082B192BCFE0D0E0CC24C394D12CBC2EF5
:1017F000C6010C2E02C0880F991F0A94E2F78023BD
:101800009123892B49F4219790F7B12C8B2DCDB7DB
:10181000DEB7E9E00C94692FB7018C2F0E946C0AA7
:101820000E948B0A019779F3F1CFCF93DF93EC01FC
:101830000E94E10BBE010E946C0A0E948B0ADF919C
:10184000CF910895983078F5863068F5E82FF0E06C
:1018500086E0989FE00DF11D11249E2F977083E084
:10186000F695E7958A95E1F7EE0FFF1FEE0FFF1F44
:10187000EE50FE4F50E040E080E0219130E0092E34
:1018800002C0369527950A94E2F721703327042E7B
:1018900001C0220F0A94EAF7822B4F5F5F4F44305A
:1018A000510559F7089580E00895983098F58630ED
:1018B00088F5E82FF0E086E0989FE00DF11D1124F7
:1018C0008E2F877041E001C0440F8A95EAF783E0CC
:1018D000F695E7958A95E1F7EE0FFF1FEE0FFF1FD4
:1018E000EE50FE4F30E020E070E05191DF011197A3
:1018F000CB01022E02C0969587950A94E2F781707B
:1019000081958527842385278C932F5F3F4F243033
:10191000310559F7089590939402809393020895A6
:1019200021E030E002C0220F331F8A95E2F72095B4
:1019300030958091930290919402822393230E9488
:101940008B0C089590911102809589238093110248
:10195000282F277069F4891759F09091A50492FFF8
:1019600007C08695869586950E94900C109211026C
:10197000089521E030E002C0220F331F8A95E2F77C
:101980008091930290919402822B932B0E948B0C56
:10199000089590933E0280933D020895FC012481B6
:1019A0002223C1F0808191810E94150C92959F7035
:1019B000963091F058F4925F9F70923058F4803FC7
:1019C00019F030F4883E30F481E008959A5FF4CF46
:1019D000843FD1F380E00895883EB0F3813FD1F792
:1019E000F3CFA6E0B0E0E7EFFCE00C94532F49837F
:1019F0005A8349815A819923A1F0222391F0CA0187
:101A00000E94E10B182F682F89819A810E94550C42
:101A100069817A81812F0E946C0A2696E3E00C94FA
:101A20006F2FCA010E94220C182FF2CFCF93DF93A1
:101A3000682F81E06A3019F06D3031F480E00E9447
:101A4000A40DDF91CF910895809108079091090727
:101A500026E0FC01A2E0B7E001900D922A95E1F7A3
:101A6000603E08F458C026E0FC0111922A95E9F77F
:101A7000C0910807D091090746E050E0BE0182E01E
:101A800097E00E9466309E0122503540892B41F13B
:101A9000C90145E0969587954A95E1F741E050E008
:101AA000BA0102C0660F771F8A95E2F7CB016091F9
:101AB000000570910105862B972BB9016B5F7F4F55
:101AC000E5E076956795EA95E1F702C0440F551F6A
:101AD0006A95E2F7842B952B90930105809300057E
:101AE0002A5F3F4F4091FF04642F70E0C9010E94BC
:101AF000302F481B463010F4240F311D211572E0A1
:101B0000370710F030E020E02E5F3A4F309309079E
:101B10002093080796CFF6E06F9FB00111246C5D0B
:101B2000794F46E050E00E945030A2CFCF93DF9330
:101B3000EC01FE018491811103C0DF91CF910895E2
:101B40000E94160D2196F5CFCF93382FE09108070C
:101B5000F0910907E250F5402091FF04622F70E0F8
:101B6000CF010E94302F281B822F332361F066E0C3
:101B70000E947B2FC82FC15010F4CF91089580E2AE
:101B80000E94160DF8CF9F01280F311D21153240FC
:101B900018F080E0F0E0E0E08E0F9F2F911D8E5F47
:101BA0009A4F9093090780930807E7CF0E94960DFC
:101BB00081E00E94A40D089580914C01882359F181
:101BC0008091A40487FF27C00E94B00B8093D101AD
:101BD00040E250E064E172E080ED91E00E94663006
:101BE000892BC1F080E2E0EDF1E0A4E1B2E00190E8
:101BF0000D928A95E1F7E091A004F091A10430974D
:101C000049F086E08093D0010480F581E02D80EDDD
:101C100091E0099508950E94B00B8093C80148E0B7
:101C200050E064E372E088EC91E00E946630892B1A
:101C300089F388E0E8ECF1E0A4E3B2E001900D92D2
:101C40008A95E1F7E091A004F091A104309711F397
:101C50000280F381E02D88EC91E0DBCF882321F036
:101C60000E94A90B0E94DC0D0895882339F0909101
:101C70003C02982B90933C020E94DC0D08950F9338
:101C80001F93CF93DF938B01EA019091B8049430B6
:101C900061F58093E9008FEF9091E800815095FD08
:101CA00006C095ED9A95F1F700008111F5CF80916E
:101CB000E80085FF1AC00E942606811111C080919C
:101CC000E80085FD06C08091E8008E778093E800EB
:101CD000F2CFF80181918F018093F100219779F77C
:101CE0008091E8008E778093E800DF91CF911F917B
:101CF0000F91089543E050E0BC0182E00E943F0E46
:101D0000089546E050E0BC0182E00E943F0E089535
:101D100040E250E0BC0182E00E943F0E0895CF9364
:101D2000DF93EC0148E050E0BC0181E00E943F0EEF
:101D300088E0FE01AEEAB4E001900D928A95E1F7E9
:101D4000DF91CF910895609148018091810480FFD7
:101D500020C08091470143E0849FC00111248F522D
:101D60009D4F539A2BB1277F3BB138605FB7F894F2
:101D7000FC01649FE00DF11D1124BF016817790774
:101D8000D1F45FBF8FE594E00197F1F700C0000048
:101D900008958091490190914A0123E0829FF001CA
:101DA0001124EF52FD4F8917A0F611821082128282
:101DB0008F5F3396F8CFFC014191CF01E8E03BB94A
:101DC000000000C047FF2BB9440F000000C000C056
:101DD00000C02BB900C0EA9591F7D0CF0F931F93A5
:101DE000CF93DF93EC0110E000E090914B0190174E
:101DF000110609F06CF40E94A30E8C8190E001960C
:101E0000817099278C83DF91CF911F910F91089555
:101E100020914901A801420F511D9A01220F331F41
:101E2000240F351F2F523D4F4C81609183048091C8
:101E3000820496959017110651F04CF0442349F016
:101E4000409184040E94AF080F5F1F4FCECF442300
:101E5000B9F340E0F7CFB0E0A0E0E1E3FFE00C949D
:101E60004A2FEC014C81042F10E09801D8010E9408
:101E700028319B01AC010E94F3304B015C01E0E290
:101E8000F0E0E01BF10BA5E5B0E0AC019B010E9486
:101E9000F3306B017C019F01DF010E94AF2F9B019A
:101EA000AC010E94FE309B01AC01280D391D4A1D7A
:101EB0005B1DC701B6010E940631F22E822F90E011
:101EC00039E23F1520F143E0249F9001112435951C
:101ED0002795122F109500E085E5E82EEF188091E8
:101EE0004B01081718F10E94A30E9C8181E09923F1
:101EF00019F0903219F48FEF8093460180914601DA
:101F0000890F8C83CDB7DEB7ECE00C94662F25E506
:101F100030E0B901681B790B9B01220F331F260F9C
:101F2000371F37FFD4CF2F5F3F4FD1CF8E2D01FD0D
:101F30008F2D20914901622F600F7727771F9B011A
:101F4000220F331F260F371F2F523D4F412F609115
:101F500083040E94AF080F5FC2CFEF92FF920F93EE
:101F60001F93CF93DF93EC018C81811109C081E035
:101F70008C831092CF0292E09093450180934401AC
:101F80008091490190914A0123E0829FF001112440
:101F9000EF52FD4F891758F110E003E060914B01BB
:101FA000161758F10E94A30E809144012091CF0290
:101FB000280F2093CF0290914501980F90934501EF
:101FC000191654F4022E000C330B40914B01415072
:101FD000550B2417350734F08195809344018130E7
:101FE00009F41C82CDB7DEB7E6E00C946C2F1182A9
:101FF000108212828F5F3396CDCFE12EF12C70E0EC
:10200000C7010E94952F20914901820F482F50E06F
:102010002091CF02022E000C330BE216F306BCF027
:1020200020914501022E000C330B2E153F057CF04C
:10203000809F900111242F523D4F40918404609164
:102040008304809182040E94AF081F5FA7CFFA012A
:10205000EE0FFF1FE40FF51FEF52FD4F11821082AC
:102060001282F3CFB0E0A0E0E8E3F0E10C944A2F55
:10207000EC018A81BB24BA9480FD02C0BB24B394D6
:10208000A0904B018C81811109C081E0B81220C061
:102090008FEF8A0D8093CE0281E08C83F12CE12CAE
:1020A00046E3942EEA14B8F00E94A30E8091CE026B
:1020B00091E0B91257C0811150C080914B018150FD
:1020C0008093CE021C82CDB7DEB7ECE00C94662F75
:1020D0001092CE02E1CF009149010E0D1F2D111D6E
:1020E000C801880F991F080F191F0F521D4FF801C3
:1020F00011821082128234E0C32ED12C812C809167
:10210000CE02880D87332CF1692D0E94872F892FED
:10211000082E000C990B8E159F0591F48091840474
:102120008C9DA0018D9D500D112455954795559579
:102130004795980160918304809182040E94AF08C2
:102140008B0CF1E0CF1AD108D1F68FEFE81AF80A1C
:10215000A9CF87FFDDCF8A0DDBCF81508093CE02E0
:10216000BC82B1CF90E0019660914B0170E00E947B
:10217000952F8093CE028C83A6CFEF92FF921F9370
:10218000CF93DF93EC0110E0EE24EA94F12C609100
:102190004B01161770F00E94A30E9A818C8190FF5C
:1021A00027C08F5F8C83DF91CF911F91FF90EF90BD
:1021B000089520914901422F410F5527551FCA010B
:1021C0009A01220F331F280F391F2F523D4F70E005
:1021D000C7010E94952F962F8C81409184046091B5
:1021E0008304199F800D11240E94AF081F5FCFCF79
:1021F0008150D8CF9091810490FF0EC090914901F9
:1022000020914A0133E0939FF0011124EF52FD4FDA
:10221000921718F00E94A30E089581836083428371
:102220009F5F3396F5CFA3E0B0E0E9E1F1E10C94D4
:10223000522F8C018091D00281110AC09E012F5F24
:102240003F4F48E76FEF0E94AF088A818093D0022A
:10225000F8016481613069F08091D00240E066232A
:1022600061F040E0623011F44091D00280E060E023
:1022700004C06091D00240E080E00E94FA10F801B2
:10228000848190E0019663E070E00E94952F848342
:102290002396E4E00C946E2FA3E0B0E0E2E5F1E1D8
:1022A0000C94542F9091810490FF0AC09E012F5FDF
:1022B0003F4F0E94AF084B8169818A810E94FA10CA
:1022C0002396E2E00C94702FCF93DF93EC01E1E8CA
:1022D000F4E0438162818C810E944C118C818F5F7C
:1022E0008C83DF91CF910895CF93DF93EC01EC8144
:1022F000F0E0EB54FC4F4491E1E8F4E0628181812D
:102300000E944C118C818F5F8C83DF91CF91089557
:10231000B0E0A0E0EEE8F1E10C944C2F7C015B0111
:102320006A0180916F0201E010E08A3010F40AE047
:1023300010E0C1E0D0E0B501C701F60109958111B7
:1023400004C021960C171D072CF4CDB7DEB7EAE0C8
:102350000C94682FCC9F9001CD9F300D300D11242F
:1023600090E080E045E34A95F1F70000019682177E
:102370009307C1F7E0CFB0E0A0E0E1ECF1E10C940D
:102380004E2F6C017B0164E670E088E70E948E2C82
:102390008C01E601EC0CFD1C17FD0BC0FE018491C5
:1023A00064E670E00E94FA2C8C012196CE15DF05C0
:1023B00099F70E94702D81E00115110509F080E068
:1023C000CDB7DEB7E8E00C946A2F80918D04909130
:1023D0008E04911103C091E089270895882369F044
:1023E00062E070E087EB94E00E94BB11811103C0B2
:1023F00080918D04089510928D0480918D04EBCF0F
:10240000CF93C0918D0480918E048823D1F00E94D7
:102410007507605A75418F4F9F4F60938904709381
:102420008A0480938B0490938C04C11108C062E0ED
:1024300070E085EB94E00E94BB11811105C0C09152
:102440008D048C2FCF91089581E080938D04F7CF78
:10245000B0E0A0E0EEE2F2E10C94462FFC016280D5
:10246000448081E08483E5EBF3E07490E4E3F4E0FE
:10247000E491C0918404C695C158D0E0CC0FDD1F13
:10248000CD2FDD27812C75E0972EAA24AA94B12C9C
:1024900055245A94E719EE2EF12C80914B018816A1
:1024A00038F00E94A30ECDB7DEB7E0E10C94622FA6
:1024B000C82CD12C82E0861568F09C9CF0019D9C74
:1024C000F00D1124ED58FC4F80918204808380919F
:1024D00083048183411023C09C9CF0019D9CF00DDE
:1024E0001124ED58FC4F1382128220914901C6013C
:1024F000820F911D9C01220F331F280F391F2F526D
:102500003D4F9C9CF0019D9CF00D1124ED58FC4F1B
:102510004281618180810E94AF088394BECF9C9CE0
:1025200080019D9C100D11240D581C4FF8018381D2
:102530008823F1F081508383859DC001112464813B
:1025400070E00E94302FFB01FF27EB54FC4F849179
:10255000E82FE719E59DC0011124B7010E94302F33
:1025600080918404689FB0011124F8017283BDCF6B
:102570000E944030B5010E94952F8C179D070CF0EA
:10258000B4CFF2E0F61598F40E944030B5010E94F5
:10259000952FF80180830E94403020918304269576
:1025A000622F70E00E94952F280FF80121839C9CD8
:1025B000F0019D9CF00D1124ED58FC4F128280918A
:1025C0008404893C58F088EC9C9CF0019D9CF00DA3
:1025D0001124ED58FC4F8483838387CF8431A0F787
:1025E00084E1F2CFB0E0A0E0E8EFF2E10C944A2FF2
:1025F00049015A016B017C010E9499088401A401E0
:102600006A2D7B2D88E090E00E94B23094014A2D23
:102610005B2DB601C70100E20E94D92F622F84E230
:1026200090E00E94A030CDB7DEB7ECE00C94662FAE
:10263000A3E0B0E0EEE1F3E10C944D2F082FE62E7D
:10264000F42EC22E9091810490FF41C0209182040B
:10265000281308C080918304861304C080918404E9
:10266000841729F08091CD0282608093CD02E92FFA
:10267000E695E695AE2FB0E0A656BE4F8C918093BE
:10268000CB029C7F943039F59E012F5F3F4F4F2D39
:102690006E2D802F0E94AF084B8169818A810E9434
:1026A000FA1000938204E0928304F0928404CC2018
:1026B00071F0209181046091850470918604302F1F
:1026C000A70180918704909188040E94F2122396BA
:1026D000E9E00C94692F823019F4F0908404E1CF82
:1026E0008630A1F1893091F18931D9F6E9516E2F07
:1026F0006170B62EE695F0E0E055FC4F1491D12CB8
:1027000060914B01D61618F00E94A30ECACFD19E3D
:10271000C001112470E00E94302F802FB11014C02E
:10272000860F20914901622F6D0D7727771F9B013E
:10273000220F331F260F371F2F523D4F4F2D6E2D67
:102740000E94AF08D394DCCF861BEBCF022FA9CF1A
:10275000E1E8F4E0438121E1421B08F440E021E09C
:10276000628181810E9418130895E1E8F4E04381B9
:1027700021E1420F08F44FEF21E0628181810E9444
:1027800018130895E1E8F4E0628121E1621B08F486
:1027900060E021E0438181810E9418130895E1E8FF
:1027A000F4E0628121E1620F08F46FEF21E04381E0
:1027B00081810E9418130895E1E8F4E0818121E00D
:1027C000438162818A500E9418130895E1E8F4E081
:1027D000818121E043816281865F0E941813089500
:1027E00080918504882319F081508093850420917D
:1027F000810430918204409183045091840460915B
:1028000085047091860480918704909188040E94C9
:10281000F212089580918504833018F48F5F8093BD
:102820008504209181043091820440918304509169
:10283000840460918504709186048091870490914E
:1028400088040E94F2120895E1E8F4E085E08083B4
:1028500011828FEF828388E783831482ABECB2E02E
:1028600012968C911297836012968C93758125E055
:1028700030E04FEF58E760E0868197810E94F212C6
:1028800008959091A50492FB222720F9281779F04A
:1028900080FB92F99093A5046091A4047091A50423
:1028A00084E090E00E94BE3082E00E94A20C089575
:1028B000A4E0B0E0EEE5F4E10C94532F4091530214
:1028C0005091540260915502709156022FB7F894BE
:1028D0008091A7049091A804A091A904B091AA04A2
:1028E0002FBF841B950BA60BB70B11E08436910507
:1028F000A105B10570F10E9461096E5F7F4F8F4F96
:102900009F4F69837A838B839C838091150190917B
:102910001601895A9D4F4091140150E045305105F0
:1029200010F044E050E0BE016F5F7F4F0E947330B3
:1029300082E090E00E94BA2E182F882351F00E9466
:1029400075076093530270935402809355029093DD
:102950005602812F2496E3E00C946F2FABE0B0E099
:10296000E4EBF4E10C94542F88E0E1E8F4E0DE01BC
:10297000119601900D928A95E1F78091CB0290918A
:10298000CC02A091CD0289879A87AB872B85409195
:102990006B0250916C0260916D0270916E023FB7B4
:1029A000F8948091A7049091A804A091A904B091F3
:1029B000AA043FBF841B950BA60BB70B8436910569
:1029C000A105B10510F4222319F180911D01909108
:1029D0001E01895A9D4F40911C0150E04C30510519
:1029E00010F04BE050E0BE016F5F7F4F0E947330EC
:1029F00083E090E00E94BA2E882369F00E94750758
:102A000060936B0270936C0280936D0290936E02E0
:102A10001092CD0281E02B96E2E00C94702FEF92A1
:102A2000FF921F93CF93DF9300D000D00F92CDB7CA
:102A3000DEB77B0190E080E00E94BA2E182F882339
:102A400009F487C04091070150E04115510511F08C
:102A500041E050E06091080170910901695A7D4F91
:102A6000CE0105960E94733040914F025091500262
:102A700060915102709152022FB7F8948091A7048F
:102A80009091A804A091A904B091AA042FBF841B1F
:102A9000950BA60BB70B84369105A105B10540F443
:102AA00088E592E00E94F0059D81891709F451C0E4
:102AB00081E090E00E94BA2E81111AC010E080914E
:102AC0004B0290914C02A0914D02B0914E02F70141
:102AD00080839183A283B383812F0F900F900F90F7
:102AE0000F900F90DF91CF911F91FF90EF9008957D
:102AF00040910F0150E04530510510F044E050E0A6
:102B00006091100170911101695A7D4FCE010196BB
:102B10000E94733088E592E00E94F0059D81891340
:102B2000CDCF0E94750760934F027093500280933F
:102B300051029093520289819A81AB81BC8180932A
:102B40004B0290934C02A0934D02B0934E0211E0C1
:102B5000B6CF8091580290915902A0915A02B0913B
:102B60005B0289839A83AB83BC831111E4CFA7CF27
:102B7000A8E0B0E0EEEBF5E10C94542F66EE7EEFAA
:102B800090E080E00E94BE3060E082E090E00E9431
:102B9000A03081E090E090933E0280933D0261E09E
:102BA00083E090E00E94A03060E074E184E090E077
:102BB0000E94BE3060E086E090E00E94A0306FEF9F
:102BC00087E090E00E94A03040E050E0BA0188E049
:102BD00090E00E94B23060E084E290E00E94A03079
:102BE00060E087E190E00E94A03060E08CE090E03F
:102BF0000E94A03060E08DE090E00E94A030198239
:102C00001A821B821C821D821E821F82188648E047
:102C100050E068E170E0CE0101960E94903040E003
:102C200050E0BA0180E290E00E94B23040E050E013
:102C3000BA018FE090E00E94B23040E050E0BA016B
:102C400083E190E00E94B2302896E2E00C94702F6D
:102C50001F920F920FB60F9211242F933F934F9311
:102C60005F936F937F938F939F93AF93BF93EF93F4
:102C7000FF938091E10082FF09C08091E20082FF12
:102C800005C08091E1008B7F8093E1008091DA00A4
:102C900080FF24C08091D80080FF20C08091DA009E
:102CA0008E7F8093DA008091D90080FF9DC080E103
:102CB00089BD82E189BD09B400FEFDCF81E080932A
:102CC000B8048091AB04811109C00E9407060E94DC
:102CD000A8068091E20084608093E2008091E10088
:102CE00080FF17C08091E20080FF13C08091E20056
:102CF0008E7F8093E2008091E20080618093E20009
:102D00008091D80080628093D80019BC85E08093C0
:102D1000B8048091E10084FF2BC08091E20084FF21
:102D200027C080E189BD82E189BD89B5982F917066
:102D300080FFFBCF8091D8008F7D8093D800809159
:102D4000E1008F7E8093E1008091E2008F7E80938E
:102D5000E2008091E20081608093E2008091B904FA
:102D6000882309F447C084E08093B8048091B804B4
:102D70008091E10083FF27C08091E20083FF23C0A0
:102D80008091E100877F8093E10082E08093B80426
:102D90001092B9048091E1008E7F8093E1008091D0
:102DA000E2008E7F8093E2008091E2008061809358
:102DB000E20042E060E080E00E9476068091F00050
:102DC00088608093F000FF91EF91BF91AF919F9148
:102DD0008F917F916F915F914F913F912F910F90C4
:102DE0000FBE0F901F90189519BC1092B804109246
:102DF000AB0474CF8091E30087FD93E09093B80417
:102E0000B5CF78941F921FB61F9211248F939F9372
:102E1000AF93BF938091A7049091A804A091A904B7
:102E2000B091AA040196A11DB11D8093A7049093AF
:102E3000A804A093A904B093AA04BF91AF919F9155
:102E40008F911F901FBE1F9018959C014FB7F8944B
:102E50008091A7049091A804A091A904B091AA041C
:102E60004FBF821B930B08952FB7F8948091A7044E
:102E70009091A804A091A904B091AA042FBF08952D
:102E80000E9434179C019091980480919904982B8A
:102E900021F0309395042093940490919A048091AA
:102EA0009B04982B21F03093930420939204E0919B
:102EB000A004F091A104309749F082E08093960439
:102EC0000680F781E02D86E994E009950895109237
:102ED0003C0280914C01882339F18091A40487FF42
:102EE00023C0E2EDF1E08EE1DF011D928A95E9F762
:102EF00090E080E00E94050890E080E00E94E007FA
:102F0000109213020E94DC0D86E0E6E9F4E0DF0196
:102F10001D928A95E9F710928F04109290041092F6
:102F200091040E9440170895EAECF1E086E0DCCFBE
:102F3000AAE2B0E0EEE9F7E10C94532F8AEB94E0BB
:102F40002091F100FC012193CF01F4E0823C9F0726
:102F5000B9F78091BB04833009F470C0B8F48130B4
:102F600009F447C0823009F4B1C08091E80083FFC2
:102F70007EC28091BA049091BB049A3008F077C267
:102F8000E92FF0E0E75CFE4C0C94A92F8A3009F49D
:102F90008CC08B3009F46FC0893039F78091BA0446
:102FA000813219F78091BE049091BF040297E8F630
:102FB0008091E800877F8093E8008091E80082FF9D
:102FC00038C09091F3008091F200029731F4809123
:102FD000F100813011F0863021F48091F10080936E
:102FE000AD048091E8008B778093E8000E9457063B
:102FF000BCCF8091BA04813A09F0B7CF8091E80044
:10300000877F8093E8008091BE049091BF04892B54
:1030100061F468E08EEA94E070E00E94030780911A
:10302000E8008B778093E800A0CF60E090E080E03C
:10303000F3CF8091B8048111C0CF97CF8091BA04AB
:10304000813A09F092CF8091BE049091BF04892B00
:1030500009F08BCF8091E800877F8093E800809112
:10306000E80080FFFCCF80914C018093F1008091BB
:10307000E8008E77B9CF8091BA04813209F075CF1C
:103080008091BE049091BF04892B09F06ECF80918E
:10309000E800877F8093E8000E9457068091BC0477
:1030A00080934C010E94671760CF8091BA048132EF
:1030B00009F05BCF8091E800877F8093E8000E9451
:1030C00057068091BD048093AC044FCF8091BA0421
:1030D000813A09F04ACF8091E800877F8093E80029
:1030E0008091E80080FFFCCF8091AC04BECF803897
:1030F00099F0823809F0BBC18091BE048F7087308F
:1031000008F0B5C18093E9008091EB0085FB88272A
:1031100080F91092E90006C08091B6049091B7043E
:10312000911182609091E800977F9093E8008093DE
:10313000F1001092F1008091E8008E7794C188230D
:1031400009F482C1823009F092C18091BC048111DE
:1031500085C18091BE048F702FEF280F263008F0B4
:1031600086C18093E9002091EB0020FF77C1933066
:1031700031F48091EB0080628093EB006FC19091FD
:10318000EB0090619093EB0021E030E001C0220F52
:103190008A95EAF72093EA001092EA008091EB000A
:1031A0008860EACF811163C11091BC041F778091C0
:1031B000E3008078812B8093E3008091E800877F93
:1031C0008093E8000E9457068091E80080FFFCCFC2
:1031D0008091E30080688093E30082E0111183E036
:1031E0008093B80444C18058823008F040C1809177
:1031F000BC049091BD048C3D23E09207A1F583E0CF
:103200008A838AE289834FB7F894DE01139620E01F
:103210003EE051E2E32FF0E050935700E49120FFAD
:1032200003C0E295EF703F5FEF708E2F90E0EA30C1
:10323000C0F0C7968D939D932F5F243159F74FBFF0
:103240008091E800877F8093E8006AE270E0CE0119
:1032500001960E9403078091E8008B778093E80035
:1032600006C1C096E7CF4091BE045091BF04292FFC
:1032700033272330310509F444C078F52130310576
:1032800009F46FC08BE390E0E3EBF5E02230310509
:1032900009F0EDC02091E800277F2093E8002091FD
:1032A000C0043091C1048217930708F49C0140E0E8
:1032B0002115310509F064C0411162C08091E80018
:1032C00082FDC9CF8091B804882329F2853019F294
:1032D0008091E80083FFF2CFBECF21323105A9F102
:1032E0002232310509F0C3C04115510509F443C02C
:1032F0004130510509F0BBC086EB90E0E9EBF4E00A
:10330000C9CF992781309105C1F0009759F00297F4
:1033100009F0ADC0E0E0F6E0E4918E2F90E0E0E04F
:10332000F6E007C0E0E2F6E0E4918E2F90E0E0E204
:10333000F6E0009709F49BC0ADCFEEE0F6E0E49133
:103340008E2F90E0EEE0F6E0F4CF4115510571F0DC
:103350004130510509F08BC089E090E0EEEDF5E0D9
:1033600099CF82E190E0EEEEF5E094CF89E090E035
:10337000E5ECF5E08FCF84E490E0EFE6F5E08ACF6E
:103380008091B804882309F466CF853009F463CFAF
:103390008091E80083FD5FCF8091E80082FD8ECFB1
:1033A0008091E80080FF84CF9091F3008091F2003B
:1033B0002115310519F08830910550F041E008974A
:1033C00009F040E08091E8008E778093E80070CFAC
:1033D00044914093F1003196215031090196E8CF94
:1033E000803809F044C08091E800877F8093E8002E
:1033F0008091B9048093F1009ECE811138C0109164
:10340000BC041230A0F58091E800877F8093E8002B
:103410001093B9040E945706112311F084E005C0EF
:103420008091E30087FDFACF81E08093B80442E009
:1034300061EC81E00E94760642E261EC82E00E944B
:1034400076068091B80413C08091BC04813079F471
:1034500081E0933009F080E08093B7041092E90096
:103460008091E800877F8093E8000E945706809152
:10347000E80083FF0AC08091E800877F8093E8001E
:103480008091EB0080628093EB00AA96E3E00C94BD
:103490006F2F1F920F920FB60F9211242F933F930D
:1034A0004F935F936F937F938F939F93AF93BF934C
:1034B000CF93DF93EF93FF93D091E900DF7080917A
:1034C000EC00C82FC17080FDC0E81092E900809127
:1034D000F000877F8093F00078940E9498171092F4
:1034E000E9008091F00088608093F000CD2BCF70D0
:1034F000C093E900FF91EF91DF91CF91BF91AF9120
:103500009F918F917F916F915F914F913F912F91FB
:103510000F900FBE0F901F9018950E9467172FEF06
:1035200084E39CE0215080409040E1F700C000001F
:1035300088E19AE00FB6F894A895809360000FBEDA
:1035400090936000FFCF4091980490919A0420914D
:103550009B04662309F469C0942B922B2091990453
:10356000922B31F098E090938F0491E09093900427
:103570008D3C41F40E945D088195809399040E94DE
:10358000401708958E3C19F40E945D08F6CF8F3CD9
:1035900031F40E945D08819580939804F0CF803DBE
:1035A00019F40E945D08F8CF893D29F40E943B0878
:1035B00080939A04E4CF8A3D21F40E943B088195D0
:1035C000F7CF8B3D31F40E943B08819580939B049B
:1035D000D6CF8C3D19F40E943B08F8CF9FE2980F9C
:1035E000983070F4815D990B21E030E001C0220F2A
:1035F0008A95EAF780919704822B80939704BFCF36
:103600008D3D31F480919104816080939104B7CF16
:103610008E3D21F4809191048260F7CF8F3D09F0B7
:10362000AECF809191048460F0CF8D3C59F48091AD
:10363000990487FF0DC01092990441110BC010929C
:103640008F0408C08E3C81F48091990418169CF375
:10365000442381F080919A0490919B04892B09F076
:103660008ECF109290048BCF8F3C49F447FFF0CF60
:1036700010929804809199048111ECCFE0CF803DA5
:1036800019F41416ACF3E4CF893D29F4191604F7A4
:1036900010929A04DDCF8A3D19F497FFD9CFF8CF65
:1036A0008B3D29F427FFD4CF10929B04D1CF8C3DC2
:1036B00019F41216CCF3CCCF9FE2980F983090F407
:1036C000815D990B21E030E0B90102C0660F771FE0
:1036D0008A95E2F7CB018095909197048923809396
:1036E0009704B6CF8D3D31F4809191048E7F809305
:1036F0009104AECF8E3D21F4809191048D7FF7CF60
:103700008F3D09F0A5CF809191048B7FF0CF882366
:1037100081F19CEF980F913A28F40E9481070E9452
:10372000DC0D089590E2980F983050F4877091E086
:1037300001C0990F8A95EAF7892F0E94A90BEFCF54
:103740009BE5980F933028F490E080E00E940508F4
:10375000089598E5980F9B3128F490E080E00E944E
:10376000E007089593E3980F933118F460E00E9406
:10377000A31A0895CF93C82F8823B1F18CEF8C0F33
:10378000813AA0F580914C01882301F18091A40435
:1037900087FF1CC0EC2FE695E695E695F0E0E05338
:1037A000FE4F828190E04C2F477021E030E002C054
:1037B000220F331F4A95E2F782239323892B79F056
:1037C0008C2F0E9481070E94DC0D09C0EAECF1E019
:1037D0008191C817A9F381E0E03DF807C9F78C2F64
:1037E0000E94AC070E94DC0DCF91089580E28C0FFF
:1037F000883068F4C77021E030E001C0220FCA951C
:10380000EAF780913C02822B80933C02EBCFEBE500
:10381000EC0FE33040F4F0E0E35BFE4F808190E09A
:103820000E940508E1CFE8E5EC0FEB3150F4F0E041
:10383000EE0FFF1FE05BFE4F808191810E94E00749
:10384000D3CF83E38C0F833178F661E08C2F0E9415
:10385000A31ACACF0F931F93CF93DF93C62FD42FF2
:10386000022FFC0185818823A9F06093FE040E9449
:1038700034179093FD048093FC04C77081E001C06D
:10388000880FCA95EAF70E94350EDF91CF911F91FC
:103890000F9108958091FE04681335C08091FC0457
:1038A0009091FD040E942517883C910560F510E277
:1038B0001D0FCD17B9F080E28C0F883040F4C7702F
:1038C00081E001C0880FCA95EAF70E942E0E1830D9
:1038D00048F481E09D2F977001C0880F9A95EAF710
:1038E0000E94350E802F0E94BA1B802F0E94871BDA
:1038F000183058F6D77081E001C0880FDA95EAF7E2
:103900000E942E0EC2CFC77081E001C0880FCA95F9
:10391000EAF7F6CF80919C04882319F00E943417AF
:1039200008950E946109CB01089560918104669514
:10393000669570E04BE050E089E391E00E945930D9
:10394000892B19F481E08093CC020E948A1C909309
:10395000C6028093C5028091CD0284608093CD021F
:1039600008959091810490FF3AC09370811138C0FE
:103970009460909381048091CD0281608093CD0208
:10398000662391F020918104309182044091830458
:10399000509184046091850470918604809187041D
:1039A000909188040E94F212609181046695669558
:1039B00070E04BE050E089E391E00E945930892BA0
:1039C000B9F00E94920881E08093C80220E0409103
:1039D000840460918304809182040E9418130895E6
:1039E0008B3210F0986AC5CF880F880F982BC1CF03
:1039F0000E94951CE8CF8091810486958695815020
:103A000009F48AE261E00E94B11C0895809181046A
:103A1000869586958F5F8B3208F081E061E00E9489
:103A2000B11C08959091810490FF09C096959695D8
:103A3000981728F0961718F40E94061D089561E063
:103A40000E94B11C0895B0E0A0E0E9E2FDE10C9411
:103A50004C2F8C01FC018481882309F467C021E08C
:103A6000408151816281738195810E94F10CEC014A
:103A7000F8019581992309F483C4818180939F0281
:103A8000808180939E0280E280933101D0939D02D9
:103A9000C0939C029E0130522115304238F4F80147
:103AA0008681807F09F45EC0FE010AC09E01305409
:103AB00021153041C8F4F8018681807FFE0109F0AC
:103AC000FF27ED33F10528F4E455FF4FE491E0932F
:103AD0003101FE01E851FC47E730F10508F042C032
:103AE000ED5BFE4C0C94A92F9E013A9521153F41A8
:103AF000D8F29E01205A32452032310550F3FE01A2
:103B0000E0CF26E241EE61EEC8010E942A1C8091BE
:103B10001102877059F0F8018581882339F080916E
:103B2000A50482FF03C082E00E94A20CCDB7DEB7DD
:103B3000EAE00C94682F27E245EE65EEE5CF26E239
:103B400041EE60EEE1CF27E245EE64EEDDCF26E206
:103B500041EE62EED9CF27E245EE66EED5CF28E200
:103B600041E0EBCF1092FE049E0130572332310525
:103B700008F020C484E090E00E948A309093A5046D
:103B80008093A404FE01E150F047E232F10520F4F5
:103B9000E65BFE4C0C94A92F8091A4048160809375
:103BA000A40495C08091A50488608093A5048FC06B
:103BB0008091A4048260F3CF8091A4048460EFCF4D
:103BC0008091A4048860EBCF8091A5048160EDCF43
:103BD0008091A5048260E9CF8091A4048061DFCF49
:103BE0008091A4048062DBCF8091A4048064D7CF4D
:103BF0000E9467178091A4048068D1CF8091A404AB
:103C00008C60CDCF8091A5048360CFCF8091A40438
:103C10008E7FC5CF8091A504877FC7CF8091A404F4
:103C20008D7FBDCF8091A4048B7FB9CF8091A404F8
:103C3000877FB5CF8091A5048E7FB7CF8091A504F3
:103C40008D7FB3CF8091A4048F7EA9CF8091A404EF
:103C50008F7DA5CF8091A4048F7BA1CF0E94671791
:103C60008091A4048F779BCF8091A404837F97CF0A
:103C70008091A5048C7F99CF8091A40482FB992721
:103C800090F921E0922790FB82F990FB83F987CF8E
:103C90008091A504982F909591708E7F892B90FB31
:103CA00081F983CF9091A404892F8F7B96FF806444
:103CB00076CF0E9467179091A404892F97FB87F90C
:103CC00080586DCF61E08EE090E00E94A03060915E
:103CD000A4047091A50484E090E00E94BE300E948C
:103CE000671715CF60E0EFCF9091A404892F8F7EE6
:103CF00094FF806154CF9091A404892F8E7F90FF10
:103D000081604DCF9091A504892F877F93FF8860B4
:103D10004CCF85E35FC38091F001811104C089E23B
:103D20000E94810759C385E3FBCF992309F434C36B
:103D3000C3303CE7D30709F4F7C008F0DAC0C11577
:103D40009CE7D90709F4E3C0C130DC4709F4F2C0AD
:103D5000F8018581C081D181882309F4F9C0CE01A1
:103D60000E94E10BF82E682FCE010E94550CBE0177
:103D70008F2D0E946C0A0E948B0AD82FC92FA82E63
:103D8000F801C580B680B2943FE0B3228091110261
:103D9000877009F1EC2CCC20F9F0892F807F8034DA
:103DA00069F080E28D0F8830B0F0892F807E8032FC
:103DB00029F4F1E0FD1778F4BB2069F08091A504A7
:103DC00082FF09C082E00E94A20C809111028770DC
:103DD000EE24E3948111E12CDC2ED2942FE0D22248
:103DE0002BE02D1508F419C1ED2DF0E0E459FE4C3F
:103DF0000C94A92F8091810480FF1EC0282F2E7F54
:103E00002093810430918204409183045091840472
:103E10006091850470918604809187049091880454
:103E20000E94F2120E9492088091CD0281608093DC
:103E3000CD020E94A30E6BCE81608093810461E06D
:103E4000869586950E94B11C62CE4BEF5CE166E0E0
:103E50007DE10E948B085BCE46E05DE16BEF7CE18B
:103E6000F8CF4CED53E166EE73E1F3CF46EE53E14C
:103E70006CED73E1EECF42EC53E16FEC73E1E9CF0F
:103E80004FEC53E162EC73E1E4CF48EA53E165EBB8
:103E900073E1DFCF45EB53E168EA73E1DACF40EF3E
:103EA00053E16AE074E1D5CF4AE054E160EF73E199
:103EB000D0CF61E081E0C6CF65E082E00E94121DB4
:103EC00026CE68E086E0FACF6EE089E0F7CF64E1C5
:103ED0008FE0F4CF67E185E1F1CF61E088E1B2CF17
:103EE00062E289E1EBCF61E083E2ACCF6AE285E296
:103EF000E5CFCB35FCE7DF0749F1CC352CE7D2071E
:103F0000D9F0CA35DC4709F023CF81E01CC00E94FC
:103F100067178FEF94E3ECE081509040E040E1F7C9
:103F200000C000000E9464076FEF7FEF90E080E028
:103F30000E94BE300E948D1A8091A50482FB8827C2
:103F400080F991E089270E94411402CF80E0FBCFE5
:103F5000CE010E94220CF82E0ACF3C2F3F70F32E88
:103F6000C07F19F0F29490EFF922CC20B9F0FF2035
:103F700069F080E28D0F883010F0A11009C08091A7
:103F80003C02F82AF0923C020E94DC0D8D2F43C0C7
:103F900080911302F82AF0921302F6CF8D2F0E941F
:103FA000871BFF20D1F1D05ED83010F0A11004C0E3
:103FB0008F2D0E94A90B06C0F09480911302F82265
:103FC000F09213020E94DC0D28C08C2F8F70F82E07
:103FD000C07FC03219F0F29480EFF822AA2059F085
:103FE00091E0A91609F479C0CC2009F485C0BB2062
:103FF00009F447C0CBCF8091A50482FD3EC0CC2000
:10400000B1F1FF2039F080913C02F82AF0923C0295
:104010000E94DC0D80E00E94BA1B2D2D2850330B2E
:104020002430310510F40E942A08EE20A9F0809176
:10403000110280FD11C0F80115828695869586953E
:104040000E94B90CC8010E94231D8091110286951F
:10405000869586950E94900C20E0F8014081518160
:1040600062817381848195810E94F10C5FCD80E033
:104070000E94871BFF2089F29BCFCC20A1F0B110BA
:1040800004C08F2D0E94350EC8CFE1E0BE12C5CF0F
:10409000809112029F2D9823F91609F4BECFF82AB9
:1040A000F0921202BACFB110B8CF8F2D0E942E0E0F
:1040B000909112028F2D892329F08F2D80958923CD
:1040C000809312028091F1019F2D982309F4A5CFCE
:1040D000F094F822F092F101A0CFCC2029F0F5E085
:1040E000FB1508F49ACFCDCF24E02B1508F495CF1B
:1040F0008F2D0E942E0E91CFBB20D1F339E3A31256
:1041000009C08FEF97EEE3E081509040E040E1F787
:1041100000C000008D2F0E94871B7FCF8C2F8695BB
:104120008695837069F0813009F077CF8D2F9C2FB1
:104130009370C11002C080E090E00E94E0076DCF54
:104140008D2F9C2F9370C11002C080E090E00E94E0
:10415000050863CF6C2D8D2F0E94A31A5ECF8C2F84
:10416000837009F03FC0C11058CF4D2F429546953E
:104170004770440F440F2D2F2F7030E0042E02C0E3
:10418000220F331F0A94E2F790E080E0D4FF09C0C9
:104190008FE090E002C0880F991F4A95E2F7809562
:1041A0009095C695C695C370C23099F078F4409149
:1041B0003D0250913E02C13039F0822B932B842373
:1041C00095230E94C90C29CF242B352B822B932BAE
:1041D000F8CF822B932B20913D0230913E02822713
:1041E0009327EFCF8695CC2011F08C2F81708823F8
:1041F00009F413CF4D2F429546954770440F440F55
:104200002D2F2F7030E0042E02C0220F331F0A948E
:10421000E2F790E080E0D4FF09C08FE090E002C0B8
:10422000880F991F4A95E2F780959095C695C69597
:10423000C370C23099F078F4409193025091940287
:10424000C13039F0822B932B842395230E948B0C51
:10425000E4CE242B352B822B932BF8CF822B932B60
:10426000209193023091940282279327EFCFCF7051
:10427000CC2029F08C2F0E94B90C8D2F03CF8D2FCD
:104280000E942E0E8C2F0E94900CC7CE8D2FF2EF25
:10429000AF1699F1FA1570F020EFA216D1F031EFB8
:1042A000A31691F0CC2009F45BC0B1106FCE8C2F17
:1042B0008F7127C093EFA91639F1E4EFAE12F2CF58
:1042C0008091A50482FD2EC08C2F8F71CC20D9F255
:1042D00018C0CC2069F0F4E0FB1508F49ECECF7135
:1042E00081E090E002C0880F991FCA95E2F7B8CF2D
:1042F00025E02B1508F491CEF2CF8C2F8F71C110D1
:10430000C2CF0E94B90C89CE90E080E0CC2009F4A5
:104310009DCFCF7181E090E002C0880F991FCA95B0
:10432000E2F794CFCC2089F0CF718C2F0E94B90C8A
:104330008091A50482FF07C038E0C39FC00111240B
:104340008360809311028C2FDCCF81E00E94A20C4D
:1043500081E08B1508F061CE82E00E94A20C5DCE58
:10436000BB2059F0893309F0D5CE9FEFE7EEF3E09B
:104370009150E040F040E1F7CBCE8C2F8F7183CF8E
:10438000FE01E851FC47E730F10508F4A9CBC6313E
:104390002CE7D20709F4BFCC80913C028272FE0167
:1043A000E052F847E531F10508F0D2CCE858FE4C70
:1043B0000C94A92FC631FCE7DF0709F0B6CC809139
:1043C0003C028A7A91E009F490E09093F001811127
:1043D000A0CC89E20E94AC070E94DC0D98CBCF9361
:1043E000DF9380911002807F09F04DC080910F0211
:1043F000882309F448C0E091FB045091C204C091A5
:104400000B02D0910A0260910C0270910D0247E0FC
:104410005E17C9F18E2F90E0E49FF0011124ED5357
:10442000FB4F2481222391F1489FF001499FF00D19
:104430001124DF01AD53BB4F11962C9111972C1312
:1044400025C02C912D1322C015962C911597211162
:104450001DC012962D913C91261B370B283C31052F
:10446000A8F4809110028F70806180931002E7534E
:10447000FB4F80818F70806180838AE092E00E9490
:10448000231D0E94D70BDF91CF910895FC01319637
:10449000E770BECFA4E1B0E0E0E5F2E20C944A2F71
:1044A0008C0186E0F801DE011F9601900D928A953D
:1044B000E1F7F8018481E5809AE0A92E92E0B92E17
:1044C00090910E02911128C0882319F1EE20F1F08D
:1044D000C8010E94CE0CF82E8823C1F087E0F801B5
:1044E000D50101900D928A95E1F780910E028130FD
:1044F00031F480910A0290910B020E94150C0E94E7
:10450000EF218F2D6496ECE00C94662FC8010E9479
:10451000231DFF24F394F5CFD080C1808280938047
:10452000F0900F0220910C0230910D02A401421B69
:10453000530BFF2009F4D9C0483C510508F092C044
:104540008823F9F290910B0280911002282F207F8E
:1045500009F056C0C91214C090910A02D91210C0B5
:10456000E11048C08F708061809310028AE092E071
:104570000E94231D80911002F8018683F12CC1CF87
:10458000E11038C06C2D8D2D0E94D1056C2D8D2D24
:104590000E94D105E82E8111F1CFDF86C88A8F8570
:1045A00098890E94150C292F22952F70243058F4D9
:1045B0009F70223088F0992399F0F8019681907FBE
:1045C00079F4FE2C9ECF2A5F2F70223068F0C8014C
:1045D0000E94231DEF2CF5CF992311F0882389F336
:1045E000805E883070F3F3CF803F58F3815F833073
:1045F00070F7E7CF80911002816080931002BECFE8
:10460000C91207C090910A02D91203C0EE2009F422
:104610008DC0C8010E94CE0C882309F477CFEE200C
:1046200009F474CF80911002803288F020910A0240
:1046300030910B02398728879B868A8690910E02DB
:104640009C871D868E87CE0108960E94231D87E0D9
:10465000F801AAE0B2E001900D928A95E1F70E947C
:10466000EF2157CF90911002292F207F51F48AE03B
:1046700092E00E94231D87E0F50111928A95E9F7E7
:104680007DCF882309F43DCF80910B028C1110C09F
:1046900080910A02D8120CC0E1100AC09683C801AA
:1046A0000E94231D87E0F50111928A95E9F729CF31
:1046B000C8010E94CE0C882309F428CFEE2009F40B
:1046C00025CF80911002803210F220910A023091A1
:1046D0000B023A8329839C828B8290910E029D83E8
:1046E0001E828F83CE010196B0CF483C5105D0F693
:1046F000882309F40ECFFE2CEE2009F407CF809119
:104700000B028C1120C080910A02D8121CC080912B
:10471000100280FD0FC0982F907F61F08683903F3C
:1047200031F0982F907F905F8F70892B8683C8011E
:104730000E94231D87E0F801AAE0B2E001900D92EB
:104740008A95E1F7DECEC8010E94CE0C81117FCFA1
:1047500080911002816080931002C8010E94231D85
:10476000D0CEABE1B0E0E7EBF3E20C94522F4E8BEE
:104770005F8B688F798F8A8F9B8F192F9111109281
:1047800013021D8A86E0FE017696DE011F960190D7
:104790000D928A95E1F70A8D002341F021E04F85C3
:1047A000588969897A89C8010E94F10C0B8B1C8B8E
:1047B00087E0FE013F96DE01189601900D928A95E2
:1047C000E1F7CE0108960E944A2281110CC087E0D1
:1047D000FE013896DE01119601900D928A95E1F75F
:1047E0008C8581110BC017E08091FB049091C2046D
:1047F000891331C06B96E4E00C946E2F2091C204B3
:1048000030E0C9010196877099274091FB04481751
:10481000190699F097E0929FD001939FB00D112453
:10482000AD53BB4FFE01319601900D929A95E1F781
:104830008093C2040E94D70BD6CF0E9467171092B4
:10484000C2041092FB0487E0EAE0F2E0DF011D926F
:104850008A95E9F7C8CF819FC00111248D539B4FE2
:104860000E944A22882331F28091FB0490E0019655
:10487000877099278093FB04B7CFA3E1B0E0E3E40E
:10488000F4E20C94492F8E01045F1F4F88E0D80199
:104890001D928A95E9F788E8C82E81E0D82EF12C80
:1048A000E12CAA24A394B12C22E9822E21E0922E9D
:1048B000F60181916F018F3F09F442C0F894E82F0F
:1048C000E295EF70F0E021A18F70A50102C0440FC6
:1048D000551F8A95E2F7CA01922F982B91A392A1B6
:1048E0008095892382A3789400C0ECE8F1E0712CD4
:1048F00031E021912F3F09F498C0A22FA295AF700B
:10490000B0E090968C9190E02F7002C095958795BD
:104910002A95E2F780FD89C0832F782A330F8E16FF
:104920009F0639F7F601319780818F3F11F00E9481
:104930004A0950EA5A95F1F7F801EE0DFF1D708211
:104940008FEFE81AF80AA4E0EA16F10409F0B0CFF4
:1049500048E050E0B80184E792E00E94663000979A
:1049600041F028E0F801A4E7B2E001900D922A9509
:10497000E1F700917D0210E001581D4F892B09F4E9
:1049800056C081E0809343020E9434179093420204
:1049900080934102F12CE0909C04EE2009F4A1C028
:1049A00019821A821B821C8280916F028A3008F061
:1049B00062C04FE055E1BE016F5F7F4FC8010E94AA
:1049C0008811882309F47CC048E554E1BE016F5F7B
:1049D0007F4FC8010E948811882309F471C04EEAF4
:1049E00054E1BE016F5F7F4FC8010E948811882388
:1049F00009F466C010926F0280917C0290E044E05E
:104A000050E0BE016F5F7F4F81589D4F0E9466301E
:104A100021E020934A02892B09F044C0E12C8E2D1D
:104A20008F296396EDE00C94652F80E076CFF090AF
:104A30004302FF2009F4AECF8091410290914202DF
:104A40000E942517059708F4A5CF44E050E064E7DD
:104A500072E0C8010E946630892B59F084E0E4E7D7
:104A6000F2E0D80101900D928A95E1F7109243028D
:104A700092CFF12CFBCF80914402909145020E948D
:104A80002517843F914008F094CF80914A028823F3
:104A900029F284E0FE013196DF011D928A95E9F743
:104AA00010924A02E0917C02F0E0E158FD4F8981CA
:104AB0009A81AB81BC8180839183A283B383AFCF82
:104AC00080916F028F3F31F08F5F80936F028A3049
:104AD00008F492CF0E9434179093450280934402C9
:104AE000D4CF84E0F801A8E5B2E001900D928A9558
:104AF000E1F788E592E00E94F005809357028090EC
:104B00005C0290905D02A0905E02B0905F02809186
:104B1000460290914702A0914802B091490288163E
:104B20009906AA06BB06B1F080924602909247020F
:104B3000A0924802B09249020E947507861A970A0D
:104B4000A80AB90A8092700290927102A092720231
:104B5000B09273028BE0E0E6F2E0DE011196019084
:104B60000D928A95E1F78091600286958695D090A6
:104B70006102C0906202B0906302009169021091DC
:104B80006A0210926A02112309F449CF10FF0BC088
:104B900029819091810420FF1AC091609093810433
:104BA00060E00E94B11C11FF06C020E04B2D6C2D6F
:104BB0008D2D0E94181312FF04C00023A9F00E943B
:104BC000951C13FF2CCF81E08093C80228CF9E7FD5
:104BD000909381040E9492088091CD02816080931D
:104BE000CD020E94A30EDFCF0E949208EACFA6E07A
:104BF000B0E0EDEFF5E20C94522F0E9434178C01D7
:104C000080913F02909140028017910781F01982B4
:104C10001A820E943417682F49815A81792F80E0C7
:104C200090E00E94B1231093400200933F02269629
:104C3000E4E00C946E2F1F921FB61F9211248F93E5
:104C40009F93AF93BF938091A604811113C080916D
:104C5000A7049091A804A091A904B091AA04419638
:104C6000A11DB11D8093A7049093A804A093A9044B
:104C7000B093AA04BF91AF919F918F911F901FBED7
:104C80001F901895CDB7DEB761970FB6F894DEBFC9
:104C90000FBECDBF85B7806885BF85B7806885BFEB
:104CA00084B7877F84BF0FB6F894A8958091600081
:104CB000886180936000109260000FBE80E890E0F1
:104CC0000FB6F89480936100909361000FBE88E462
:104CD00099E09093C7018093C6010E9407060E9445
:104CE000A8068091E20084608093E200789480912D
:104CF000B8048823A1F01091E9001F709091EC0096
:104D0000892F817090FD80E8182B1092E900809126
:104D1000E80083FD0E9498171F701093E90082E05D
:104D200084BD93E095BD9AEF97BD80936E0010927D
:104D300070021092710210927202109273028091AE
:104D4000D80080618093D8002AE12A95F1F700C04D
:104D50008091D900182F117080FD04C00E940706B1
:104D60001092B80410939C0410939D041093240196
:104D7000112309F472C0109247018BE1809348011E
:104D80000E94CE2D809124018091240194E0811114
:104D900090E090937D0284E0891B80937C0284E9FB
:104DA0000E944A0986E60E944A0987E90E944A0948
:104DB00086EC0E944A090CE811E0D8018D918D0122
:104DC0008F3F11F00E944A09B1E002391B07A9F791
:104DD00088E0EFE7F2E0DF01282F1D922A95E9F73E
:104DE000E4E7F2E0DF011D928A95E9F790E080E0C8
:104DF0000E948A30863E9E4F11F00E94B81582E0D4
:104E000090E00E947C308093870284E090E00E94D2
:104E10008A309093A5048093A4040E943D24EFEF70
:104E2000F6E721E0E150F0402040E1F700C000004B
:104E30000E943D2480919D04E4E08111E0E0F0E0D7
:104E4000E158FD4F808181FF0EC06FEF7FEF90E052
:104E500080E00E94BE300E9464078BE1809347018E
:104E6000809348018FCF83E090E00E947C3090E0F7
:104E70000E94C90C80919C04811133C182E080930F
:104E8000C00280E88093FF040E94882C6BE070E0F1
:104E90008FE192E00E94BB118823E9F18091C0026A
:104EA00065E070E081FD1FC18AE192E00E94BB11C4
:104EB000882389F16DE070E088E092E00E94BB11E8
:104EC000882349F10E947507605A75418F4F9F4FA3
:104ED0006093890470938A0480938B0490938C046C
:104EE000E2E0F5E080E092E0DF019C011D922150BC
:104EF0003040E1F7F0930907E09308078FEF9FEF49
:104F0000909301058093000581E080938E04809347
:104F10008D041092C10280917E0281117CC090E0CC
:104F200080E00E948A30863E9E4F21F00E94B81594
:104F30000E94241488E090E00E9484304B015C01C0
:104F400084E290E00E947C30282F30E040E050E086
:104F500060E070E080E090E000E20E94BE2F28292F
:104F600039294A295B292093810430938204409394
:104F70008304509384046093850470938604809323
:104F80008704909388048091CD0283608093CD0242
:104F90002C7F89F50E94241488E090E00E948430E0
:104FA0006B017C0184E290E00E947C30282F30E08D
:104FB00040E050E060E070E080E090E00E94BE2FB2
:104FC000B22FA32FF42FE52F5B0197018601BC2997
:104FD000A12BFE29E32BB0938104A0938204F093CC
:104FE0008304E093840460938504B09286048093E4
:104FF0008704909388040E9499080E9492088091E7
:10500000810480FF05C060E0869586950E94B11CF2
:1050100081E080937E0280919C04811102C00E94F5
:10502000D12D85E291E09093A1048093A004AAE0A1
:105030008A2E912CA12CB12C8091B80400E112E1B0
:10504000853009F48DC00E943D2408E812E0FFE796
:10505000EF2EF2E0FF2ED701F80191918D9132E011
:10506000E039F30709F486C09817B9F340909C041F
:10507000D12C33243394D701CD907D01F801519088
:105080008F015C1429F15C24712C66246394852DB6
:105090008621B1F04420A1F07F82D8860E94341787
:1050A0009A8789873B8691E08C2D862109F490E0D0
:1050B0009C874F81588569857A858B850E94B123AD
:1050C0007394660CF6E07F12E2CFF8013197C0824C
:1050D000D39428E0D212CFCF0E94610931E03D87FE
:1050E0004EC080E0CCCE85E192E0E0CE8091B80465
:1050F000843031F10E94E5111092A60488E190E01D
:10510000A0E40FB6F894A895809360000FBEA0931A
:10511000600083B7817F846083BF83B7816083BF72
:105120007894889583B78E7F83BF0FB6F894A8953F
:1051300080916000886180936000109260000FBED3
:105140008091B704882361F00E943D24EFE7F2E0EC
:1051500081918111B8C327E832E02E173F07C1F7CC
:105160008091B804853009F4C1CF0E9467170E946E
:105170002A0869CF98137ACF0E94F7251D8680915F
:10518000CC02882309F465C08091CB02E0918104B0
:10519000E695E695E81BE093C702823009F0B0C0BF
:1051A000F0E0E55CFD4FE4910E2F10E0E4E7EE2E19
:1051B000E1E1FE2E8091C802882361F01092C802BE
:1051C0000E948A1C9093C6028093C5021092CA0264
:1051D0001092C9020E948A1CE091C502F091C60299
:1051E0009C012E1B3F0B2F3F3F4798F520919202C9
:1051F0002223B1F0109292022091900230919102FC
:10520000821B930B8F3F9F4758F4205D3A483093A1
:105210009102209390028091CD0288608093CD020C
:10522000C090C902D090CA02E00FF11FF093C602ED
:10523000E093C50285EC92E0F70109958091C902DF
:105240009091CA02892B29F4CD2819F081E080932E
:10525000920280918E04882309F421C18091C202B8
:105260009091C3020E942517C29708F4F8C00E94CB
:1052700034179093C3028093C20282E095E090932A
:1052800009078093080780919C04882309F430C2A1
:1052900080E692E00E94960D209193023091940254
:1052A000832F9927009709F497C09C0188E0A901F2
:1052B000F4E056954795FA95E1F74115510511F03F
:1052C0008C5F9A01A90156954795569547954115CA
:1052D000510511F08E5F9A0136952795232B09F021
:1052E0008F5F813009F4BEC1882309F477C0823012
:1052F00009F4BBC1833009F4BBC18FE392E070C0F5
:10530000863059F4F0E0E85CFD4FE4910E2F10E098
:1053100074E6E72E71E1F72E4DCF893061F4E69502
:10532000F0E0EB5CFD4FE4910E2F10E06DEBE62E0C
:1053300060E1F62E3FCF8F3061F4E695F0E0EE5C51
:10534000FD4FE4910E2F10E052E3E52E50E1F52ED3
:1053500031CF853159F4F0E0E15DFD4FE4910E2F3E
:1053600010E04DEAE42E4FE0F42E24CF08E210E0E6
:105370009BE2E92E9FE0F92E883109F41BCF83329E
:1053800049F4EDE2F2E00591149133E1E32E31E1CD
:10539000F32E10CF8432C9F000ED17E0B1E9EB2E07
:1053A000B8E0FB2E853209F005CF8E2F63E00E9416
:1053B0007B2FE92FF0E0E65DFD4FE4910E2F10E02A
:1053C00028E2E22E22E1F22EF5CE04EF11E08EEE7D
:1053D000E82E8EE0F82EEECE80E069CF88E592E0F0
:1053E0000E94D60D80919F02805D0E94160D8EE670
:1053F00092E00E94960D80919E02805D0E94160DA3
:105400008AE692E00E94960D40909C0250909D0288
:1054100080912F01909130014816590609F02BC157
:1054200080919B02803209F026C1E5E9F2E08F010C
:1054300081918032E1F3F80101900020E9F79F01AA
:105440002150310979010E151F0508F44BC188E67A
:1054500092E00E94960D809131010E94160D80917C
:10546000000590910105892B09F047C180918D04B9
:105470008823A9F00E9475070091890410918A047D
:1054800020918B0430918C04601B710B820B930B69
:105490006F3F7F4F8F4F9F4710F40E94E5114D855E
:1054A00041110E94001286E0E6E9F4E0DE01119667
:1054B00001900D928A95E1F7D0909704009198049D
:1054C000F0909904E0909A0410919B041092980433
:1054D0001092990410929A0410929B04802F8F29A5
:1054E00009F445C080919404909195040E94251779
:1054F0009C0190918F04992309F405C2253131054F
:10550000B0F19F3F19F09F5F90938F04002359F0F3
:105510000E945D089FEF10160CF491E0899F802D8A
:10552000112480939804FF2059F00E945D0891E0B7
:105530001F140CF09FEF899F802D112480939904F4
:1055400080919804882399F0C0909904CC2079F038
:105550000E947D08882309F4AEC1809398048C2DA5
:105560000E947D08882309F4A8C1809399048E2D98
:10557000812B09F445C080919204909193040E947C
:1055800025179C0190919004992309F4B7C1213506
:105590003105B0F19F3F19F09F5F90939004EE208A
:1055A00059F00E943B089FEF1E140CF491E0899F74
:1055B000802D112480939A04112359F00E943B08F6
:1055C00091E011160CF09FEF899F802D112480939C
:1055D0009B0480919A04882399F0E0909B04EE202C
:1055E00079F00E947D08882309F469C180939A04A8
:1055F0008E2D0E947D08882309F463C180939B044B
:10560000809197048D1117C080919804882311F020
:10561000801311C020919904222311F02F110BC087
:1056200090919B04992311F0911305C030919A0435
:10563000332309F45EC10E94401786E0FE013196D3
:10564000A6E9B4E001900D928A95E1F70E942A083C
:105650009091C402891709F4EFCC8093C4020E9490
:105660007507EACC82E592E0BBCE8CE492E0B8CE3E
:1056700085E492E0B5CE5092300140922F0180E255
:1056800080939B02712C612C10929A0255E9C52ED1
:1056900052E0D52E60E9E62E62E0F62E8601C301C7
:1056A000B201A50194010E940631605D603319F4D6
:1056B000C016D10631F0411451046104710409F49B
:1056C00060E2D80114966C93C301B201A501940164
:1056D0000E94063129013A0101501109E016F10634
:1056E000F1F6A3CED8018D918D010E94160DABCE9F
:1056F00080E792E00E94960DB2CE80918E048823BE
:1057000009F4B4CE8091C1028111B0CE0E94001282
:1057100020910005309101052115310509F4A6CE2F
:1057200080E041E050E0482E512C1A01082E02C0C2
:10573000220C331C0A94E2F7B10162237323672B16
:1057400011F48F5FF0CF9091C00290FF9AC0880F44
:10575000880F880F8093340110923701895F8093FE
:10576000350183E08093380124E630E047E050E0E3
:1057700062E371E088E70E94282D892B09F076CE3C
:1057800095E0440C551C9A95E1F78091C00280FF8A
:105790008AC0E0EAF2E080E2DF011D928A95E9F733
:1057A000E6E9F1E0F98BE88B42E951E087E0E82E89
:1057B000DD24D394A889B9896D91B98BA88BFA019E
:1057C0008191AF01840D952D911D9C012E5F3A4F63
:1057D0003F872E87E62FF0E0E056FD4F90E080E017
:1057E0006E2C681AFD2C082E01C0FF0C0A94EAF7F3
:1057F0006E857F8500E0DB011D91BD011F21262DF7
:10580000201B2770C22E022E000C330BB12F01C0BB
:10581000BB0FCA94EAF7CB2E319521953109277039
:10582000332701C016952A95EAF7C12A1081C12AAB
:10583000C0820F5F0830F9F60196319688309105E5
:1058400079F6E889F989EA59F14009F0B3CF04E61D
:1058500010E020E230E040EA52E060E488E70E9495
:10586000492D892B09F002CE2094309480910005B7
:1058700090910105282239223092010520920005DD
:10588000F5CD8295880F807680933401920136950C
:1058900027953695279520933701815E80933501B2
:1058A0002093380161CFA2014E5F5A4F04E610E009
:1058B00020E230E0D2CF81E050CE81E056CE81E0D0
:1058C00095CE81E09BCE09BD19BD09B400FEFDCF88
:1058D0008091D8008F7D8093D8008091E000826015
:1058E0008093E0008091E00081FDFCCF0E9467176B
:1058F00037CC822B892B09F4A0CE9DCE2B303105DD
:1059000008F04ACE7DCE2B30310508F0FCCD2FCEED
:105910001092B9008CE08093B8000895B0E0A0E048
:10592000E4E9FCE20C944B2FB82EEB010E943417F3
:105930006C01EE24E394F12CC431D10560F025E034
:10594000E22EF12CCF3FDC0731F0CE0164E170E0B4
:105950000E94302F7B0184EAA82E94E8992E1092A1
:10596000BC00A092BC000E9434178C018091BC0046
:1059700087FF0DC08091B900887F8830F9F0809151
:10598000B900887F8031D1F00FEF1FEF08C0C80148
:105990000E942517E816F90648F70EEF1FEFCF3FD4
:1059A000DC07E9F2C6010E942517C817D907B8F627
:1059B000C801CDB7DEB7EBE00C94672FB092BB0007
:1059C0009092BC000E9434178C018091BC0087FF2C
:1059D0000AC08091B900887F883111F08034A1F627
:1059E00010E000E0E5CFC8010E942517E816F9068F
:1059F00060F7D3CF0F931F93CF93DF93EB01809387
:105A0000BB0084E88093BC000E9434178C01809115
:105A1000BC0087FF11C02091B900287F81E090E091
:105A2000283211F490E080E0919581959109DF9101
:105A3000CF911F910F910895CF3FDC0741F3C8012B
:105A40000E942517C817D90710F78EEF9FEFEFCFE9
:105A5000B0E0A0E0EEE2FDE20C944E2F6B018A0173
:105A60007901B9010E948E2CE6010C0D1D1DC01795
:105A7000D10711F097FF08C024E92093BC00CDB7EF
:105A8000DEB7E8E00C946A2FB70189910E94FA2CE6
:105A9000EECFB0E0A0E0EFE4FDE20C944E2FC62F75
:105AA0006A017901B8010E948E2C97FD0CC0B801E3
:105AB0008C2F0E94FA2CE601EC0CFD1CCE15DF05A4
:105AC00011F097FF08C024E92093BC00CDB7DEB7E2
:105AD000E8E00C946A2FB80189910E94FA2CEECF6D
:105AE00084E98093BC0008958EE14A9B02C08150F6
:105AF000E1F74A9BFECF08955A9880E28A95F1F724
:105B00005A9A0895FC013BE03A95F1F798E020E0BD
:105B100080E031E040E14A95F1F7880F4A9B02C0EE
:105B20008160232742E04A95F1F7000040E14A9561
:105B3000F1F7915079F790E19A95F1F799B132E048
:105B40003A95F1F7000040E14A95F1F792FB992769
:105B500090F992272081920F90830895A1E0B0E000
:105B6000E4EBFDE20C94502F19828C017C01E60ECF
:105B7000F11C0E151F0541F481E09981911180E01F
:105B80002196E6E00C946C2F0E94742DCE010196B4
:105B90000E94822DF80181938F01EBCF529A5A9A7D
:105BA000089552985A9AEA9AE9E6F0E080818F7C4B
:105BB000808308956150770B91E001C0990F6A9539
:105BC000EAF720E031E0911108C0222391F05A9ABF
:105BD00080E28A95F1F75A980895492F482339F0C1
:105BE0005A9A232740E24A95F1F79695ECCF5A98B6
:105BF000F9CF5A98EDCFFF920F931F93CF93DF9376
:105C0000EC018C01060F111DC017D10729F4CDB787
:105C1000DEB7E5E00C946D2FF9900E947C2D68E0D2
:105C20008F2D0E94DA2DF0CF1F920F920FB60F9298
:105C300011240F931F932F933F934F935F936F9371
:105C40007F938F939F93AF93BF93EF93FF93CF93E4
:105C5000DF930F92CDB7DEB719820E94742DCE016B
:105C600001960E94822D082F069506950695282FED
:105C700022952570902F9570290F922F937026955D
:105C80002695920F982797708981982B09F05CC010
:105C9000053008F059C080E18A95F1F75A9A529A76
:105CA00082E08A95F1F700C05A9888E0089F800149
:105CB0001124D801AC5FBE4F1696ED91FC91179759
:105CC0003097A9F0609186017091870114962D910B
:105CD0003C911597260F371F11968D919C91129725
:105CE000680F791F13964C9113978C910995F801C1
:105CF000EC5FFE4F6381662351F020918601309165
:105D0000870184819581820F931F0E94FB2D0E9441
:105D10007C2D80E18A95F1F75A9852985A9A80E141
:105D20008A95F1F7F801EC5FFE4F6081662351F030
:105D3000209186013091870181819281820F931F8A
:105D40000E94AE2D0E94742D0F90DF91CF91FF9194
:105D5000EF91BF91AF919F918F917F916F915F91E3
:105D60004F913F912F911F910F910F900FBE0F9068
:105D70001F9018950F931F93CF93DF93EC01059716
:105D80000CF04CC0F894529A5A9885E08A95F1F735
:105D900000009C2F969595708C2F8570980F892FF9
:105DA00083709695969523E0CC0FDD1F2A95E1F739
:105DB000980F8E01092B0E947C2D00C068E0802F77
:105DC0000E94DA2D80E18A95F1F752985A9A4A9BFF
:105DD0001EC087E090E04A991CC0FE01EC5FFE4FB8
:105DE00063816623F9F020918601309187018481D7
:105DF0009581820F931F0E94AE2D811113C0529A7C
:105E00005A9A7894DF91CF911F910F91089500C015
:105E1000DECF019729F4529A5A9A789480E0F2CF13
:105E200000C0D9CF0E94742D80E28A95F1F75A986C
:105E3000529A80E18A95F1F7CC5FDE4F6881662344
:105E400051F0209186013091870189819A81820FDA
:105E5000931F0E94FB2D0E947C2D789481E0D2CF6D
:105E6000AA1BBB1B51E107C0AA1FBB1FA617B70780
:105E700010F0A61BB70B881F991F5A95A9F780959C
:105E80009095BC01CD0108952F923F924F925F9261
:105E90006F927F928F929F92AF92BF92CF92DF923A
:105EA000EF92FF920F931F93CF93DF93CDB7DEB79F
:105EB000CA1BDB0B0FB6F894DEBF0FBECDBF099433
:105EC0002A88398848885F846E847D848C849B848A
:105ED000AA84B984C884DF80EE80FD800C811B8198
:105EE000AA81B981CE0FD11D0FB6F894DEBF0FBEC7
:105EF000CDBFED010895991B79E004C0991F961755
:105F000008F0961B881F7A95C9F78095089587FB3E
:105F1000082E062687FD819567FD61950E947B2FDF
:105F20000EF4919507FC8195089597FB072E16F4C2
:105F3000009407D077FD09D00E94302F07FC05D0D0
:105F40003EF4909581959F4F0895709561957F4F90
:105F50000895EE0FFF1F0590F491E02D09940E9423
:105F60002831332312F48A1B9B0B0C94B92F0E9407
:105F70002831B7FF0895821B930B0895002E083037
:105F800090F0982F872F762F652F542F432F322F85
:105F900022270850F4CF220F331F441F551F661FBE
:105FA000771F881F991F0A95B2F7002D089597FD56
:105FB0001094002E083098F00850232F342F452FCE
:105FC000562F672F782F892F912DF4CF1594979501
:105FD00087957795679557954795379527950A95AE
:105FE000AAF71124002D08958F929F92AF92BF922D
:105FF000CF92DF92EF92FF92CF93DF93EC01688113
:1060000079818A819B81611571058105910521F452
:1060100064E279ED8BE597E02DE133EF41E050E06C
:106020000E94D43049015A019B01AC01A7EAB1E4B6
:106030000E94F3306B017C01ACEEB4EFA50194013A
:106040000E940131DC01CB018C0D9D1DAE1DBF1DD9
:10605000B7FF03C00197A109B04888839983AA8339
:10606000BB839F77DF91CF91FF90EF90DF90CF9030
:10607000BF90AF909F908F9008950E94F42F089545
:1060800080E091E00E94F42F0895B0E0A0E08093BA
:10609000000190930101A0930201B09303010895C0
:1060A000FB01DC0102C005900D9241505040D8F731
:1060B0000895FC014150504030F001900616D1F790
:1060C0003197CF010895882799270895FB01DC01B6
:1060D00004C08D910190801921F441505040C8F7BF
:1060E000881B990B0895FB01DC0102C001900D9201
:1060F00041505040D8F70895F999FECF92BD81BD27
:10610000F89A992780B50895A6E1B0E044E050E000
:106110000C94C630A8E1B0E042E050E00C94C630E8
:10612000DC01A40FB51F4150504048F0CB01840F53
:10613000951F2E910E94A13041505040D0F70895F4
:10614000262FF999FECF92BD81BDF89A019700B430
:10615000021639F01FBA20BD0FB6F894FA9AF99AD0
:106160000FBE08950396272F0E94A1300E94A030F1
:10617000252F0E94A130242F0C94A1300196272FA7
:106180000E94A1300C94A030DC01CB01FC01F999F4
:10619000FECF06C0F2BDE1BDF89A319600B40D9273
:1061A00041505040B8F70895052E97FB1EF4009417
:1061B0000E94EB3057FD07D00E94063107FC03D048
:1061C0004EF40C94EB3050954095309521953F4F0F
:1061D0004F4F5F4F089590958095709561957F4FD3
:1061E0008F4F9F4F08950E942831A59F900DB49F17
:1061F000900DA49F800D911D11240895B7FF0C945C
:10620000F3300E94F330821B930B0895A1E21A2E03
:10621000AA1BBB1BFD010DC0AA1FBB1FEE1FFF1F4A
:10622000A217B307E407F50720F0A21BB30BE40B9A
:10623000F50B661F771F881F991F1A9469F76095E1
:106240007095809590959B01AC01BD01CF0108959B
:10625000A29FB001B39FC001A39F700D811D1124A7
:10626000911DB29F700D811D1124911D0895F89408
:10627000FFCF77189F18371A9F18371AD218F318BC
:10628000371AF019FD199F1DA31D811D9B1DA71D08
:10629000AB1DAF1D061E7B1E0E1ED81DDC1D121E63
:1062A000E01D161E221EEC1D741EF01D261EF41D80
:1062B0002A1E521EF81D2E1E591EFE1D341E3C1E87
:1062C000E41D1A1EE81D1E1E021E381E481E621EF8
:1062D000721ED21D0A1E821EAD1FAD1FE51FE51FD7
:1062E0008E20AA200D200D20AF20372146214621E7
:1062F000FA1E251F2C1F311F361F3B1F401F451F35
:106300004A1F4F1F541F591F5C1F611F641F671FC7
:0A6310006A1F6D1F701F731F761FB8
:10631A00010000000000000100000000000000046D
:10632A000100000004050000000000000B09000045
:10633A00000000000161078F0E880E810E7A0EFFA1
:10634A0000200021007F22000301191A1B1C1D1EB8
:10635A001F20212201020100360036360181828384
:10636A00E200E900EA00B500B600B700CD008301FB
:10637A00CC008A01920194012102230224022502FF
:10638A00260227022A02B300B4006F0070009F01A0
:10639A00CB019F02A0025702946697C6F4F5F6F75E
:1063AA003133000810181810080000010202020216
:1063BA000606060909090909090F0F0F0F0F0F151C
:1063CA00151518191919191919191919192324251B
:0663DA0025252525250004
:00000001FF
